:100000000C9465000C948D000C948D000C948D0064
:100010000C948D000C948D000C948D000C948D002C
:100020000C948D000C948D000C948D000C94C908D8
:100030000C948D000C948D000C948D000C948D000C
:100040000C94A8110C948D000C94B2130C94001411
:100050000C948D000C948D000C948D000C948D00EC
:100060000C94250B0C948D00000000002400270048
:100070002A0000000000250028002B0000000000DE
:1000800023002600290004040404040404040202DA
:100090000202020203030303030301020408102007
:1000A0004080010204081020010204081020000012
:1000B0000007000201000003040600000000000029
:1000C00000007401C1095D0E6C1511241FBECFEF35
:1000D000D4E0DEBFCDBF11E0A0E0B1E0E6EBFDE291
:1000E00002C005900D92A03EB107D9F714E0A0EE32
:1000F000B1E001C01D92A636B107E1F710E0CAECED
:10010000D0E004C02297FE010E94D516C23CD10760
:10011000C9F70E94C2150C94D9160C940000FB017B
:10012000DC014150504048F001900D920020C9F789
:1001300001C01D9241505040E0F70895FC0181E05C
:1001400090E00190061609F4CF010020D1F7019745
:100150000895FB0151915523A9F0BF01DC014D9198
:1001600045174111E1F759F4CD010190002049F004
:100170004D9140154111C9F3FB014111EFCF81E0D1
:1001800090E0019708950F931F93CF93DF93B82FBB
:10019000833008F075C090E00196A82FAA0FAA0F2F
:1001A000AA0F0197A53108F0A4E1482F440F440F8E
:1001B000440F71E050E0C62FD0E001E010E01EC017
:1001C000842F82508231C0F4242F30E0F901E851AD
:1001D000FE4F8081823080F4572BF901EE0FFF1F14
:1001E000E150FE4F11821082872F90E08C239D23D7
:1001F000892B11F011830083770F4F5F4A1700F3AB
:10020000BB2361F4852F8C7FF8942BB1982F9095A8
:1002100092238623982B9BB9789432C0B13009F58C
:10022000F89495B1852F8F7380958923962F9F73AE
:100230009523892B85B948B1252F30E0862F90E092
:100240002823392386E0359527958A95E1F752953D
:1002500056955695537050955423522B58B978940F
:100260000FC0852F8F70F89428B1982F990F990F90
:10027000909592238623880F880F982B98B97894AD
:10028000DF91CF911F910F910895482F863018F577
:100290002091E0013091E101672B81F481E090E051
:1002A00002C0880F991F4A95E2F780959095282300
:1002B00039233093E1012093E001089581E090E03B
:1002C00002C0880F991F4A95E2F7282B392B3093EB
:1002D000E1012093E0010895833028F4E82FF0E055
:1002E000EE51FE4F60830895CF93DF93CAE6D2E0CC
:1002F000CE010E944007239682E0CE38D807C1F78E
:10030000DF91CF9108950F931F93CF93DF938B01CC
:10031000843178F5C82FD0E0FE01E851FE4FE0812E
:10032000E33091F0E43029F582508C30E0F49E0106
:1003300022503040C901880F991F820F931F8659A0
:100340009D4F0E94DB070FC0833051F0853041F094
:10035000863031F0893021F08A3011F08B3019F479
:10036000B8010E94BE12CC0FDD1FC150DE4F1983B1
:100370000883DF91CF911F910F910895AF92BF92A3
:10038000DF92EF92FF920F931F93DF93CF930F9221
:10039000CDB7DEB7D82E7B01082F10E0F801E85169
:1003A000FE4F8081863061F480916702882341F09E
:1003B0006630710529F0109267028FEF8093B801C3
:1003C0009D2D925099839C30B8F4E4E0EE16F10430
:1003D00099F0C80102975C01AA0CBB1CA80EB91EBB
:1003E0008AE692E0A80EB91EC5010E94C9078823BB
:1003F00019F0C5010E945A074D2D4E504630B8F4F1
:100400002091E0013091E10192E0E916F10409F058
:10041000E0C081E090E0042E02C0880F991F0A948A
:10042000E2F7282B392B3093E1012093E001E98199
:10043000E23130F5ED2DE695E695E69598012770C9
:100440003070E114F10471F4F0E0E450FE4F81E00B
:1004500090E002C0880F991F2A95E2F72081282B8F
:1004600020830EC0F0E0E450FE4F81E090E002C037
:10047000880F991F2A95E2F7809520818223808337
:10048000F801EE0FFF1FE150FE4F11821082F2E0E3
:10049000EF16F104E1F083E0E816F1044CF4E11406
:1004A000F10439F191E0E916F10409F08BC032C092
:1004B000E4E0EE16F10409F45DC0F4E0EF16F10497
:1004C000CCF186E0E816F10409F07CC070C046303B
:1004D00008F08CC09981923140F48D2D60E00E942B
:1004E0001E138D2D60E00E945D1308511E4F82E0A7
:1004F00066C0F981F23108F079C08D2D60E00E946C
:100500001E138D2D60E00E945D1308511E4FF801EF
:1005100010826CC0F981F23108F068C08D2D60E066
:100520000E945D138D2D61E00E941E1308511E4F25
:1005300081E045C0F3E0DF1681F085E0D81669F070
:1005400096E0D91651F0E9E0DE1639F0FAE0DF1650
:1005500021F08BE0D81609F049C08D2D61E00E9492
:100560001E138D2D60E070E00E94BE1208511E4FD8
:1005700083E025C0F981FC30C8F5F801E851FE4F51
:1005800084E08083C80102977C01EE0CFF1CE80E1A
:10059000F91E8AE692E0E80EF91EC7010E94C9071B
:1005A000882321F5C701B8010E94C2081FC09EEE32
:1005B000D90EE1E0ED15D0F008511E4F86E0F801AC
:1005C000808314C084E793E060E071E00E94E60E4F
:1005D0000DC081E090E0042E02C0880F991F0A949C
:1005E000E2F780959095282339231DCF0F90CF9166
:1005F000DF911F910F91FF90EF90DF90BF90AF9030
:1006000008951F9380916702882329F01092670252
:100610008FEF8093B8011092E2011092FC011092CA
:10062000E5011092E3011092FD011092E601109293
:10063000E4011092FE011092E70110E0812F8E502C
:10064000863020F4812F62E070E003C0812F61E0EA
:1006500070E00E94BE011F5F143181F71092E1012A
:100660001092E0011F9108950F931F9304E713E088
:10067000C80161E171E042E023E00E94E10FC8019E
:1006800060EE43E851E00E94170EC80160E943ECB8
:1006900050E00E94170EC80160EC45E451E00E9452
:1006A000170EC80160ED4CE651E00E94170EC8011C
:1006B00064EF4EEB51E00E94170EC80160EF4EED63
:1006C00054E00E943B0EC8016FEF41E053E00E94EE
:1006D000350EC80140E051EE60E070E00E94561017
:1006E0000E9401031F910F9108951F9310E0812F25
:1006F0008251823028F4812F66E070E00E94BE01B2
:100700001F5F1431A1F781E0809367028AEF92E0C6
:100710000E94610A1F9108951F93CF93DF93282FA2
:10072000162FC82FD0E0FE01E450FE4F8081182321
:10073000442331F4FE01EB51FE4F8081811751F0CB
:1007400084E793E0622F412F50E00E94A60DCB5129
:10075000DE4F1883DF91CF911F9108958091E201C0
:10076000882349F069B18091FC0168236C7F80E0A7
:1007700040E00E948C038091E301882379F083B1EB
:1007800066B16295660F660F607C8F73682B8091EF
:10079000FD01682381E040E00E948C038091E40128
:1007A000882379F086B190E08C7390709595879549
:1007B000959587956091FE01682382E040E00E9454
:1007C0008C030895EF92FF920F931F93CF93DF93C3
:1007D000F82EEB01E42E8FEF6F3F780719F4C0E09D
:1007E000D0E016C08AEF92E06F2D0E9487098AEF51
:1007F00092E06C2F0E94090A8AEF92E00E944C0A54
:100800008091680290916902009711F00E9457123E
:100810008AEF92E06F2D4E2D0E945D0A0E2D10E0A2
:100820008AEF92E00E9491090817190791F4F0925B
:100830004702C0934802C9E4D2E00C0F1D1F05C057
:100840008AEF92E00E949A098993C017D107C1F7F5
:1008500012C08AEF92E00E949109801791072CF450
:1008600084E793E065E271E004C084E793E06DE41F
:1008700071E00E94E60E82E0E80E84E793E067E70D
:100880004E2D27E432E00E94D80DDF91CF911F91C9
:100890000F91FF90EF900895AF92BF92CF92DF92A9
:1008A000EF92FF920F931F93CF93DF930E94AE03BB
:1008B00004C084E793E00E94320F84E793E00E9433
:1008C0007F0D892BB1F70E94F0116093270270937E
:1008D00028028093290290932A02A0902B02B090C4
:1008E0002C02C0902D02D0902E022091B6013091A2
:1008F000B70179010027F7FC0095102F6A197B09D1
:100900008C099D09E616F7060807190708F04BC081
:10091000EA0CFB1C0C1D1D1DE0922B02F0922C0218
:1009200000932D0210932E02C8EED1E012EF163084
:10093000C0F488818230A9F48091E0019091E101B6
:10094000012E02C0959587950A94E2F780FF09C0B1
:10095000812F0E949C12AC0184E793E0612F0E94DA
:100960008B0D1F5F2196163011F78091B80187FD1E
:100970001AC010E00EC0F901EE0FFF1FE20FF31FC7
:10098000E15DFD4F6181808170E042810E94E20360
:100990001F5F212F30E08091B801992787FD909546
:1009A0008217930744F7DF91CF911F910F91FF902A
:1009B000EF90DF90CF90BF90AF900895BF92CF920D
:1009C000DF92EF92FF920F931F93CF93DF93162F37
:1009D000EA018F3609F44FC1803750F48B3609F4A1
:1009E0006AC18D3609F4D3C1893609F03FC222C2EB
:1009F000863769F0873720F4803709F037C2E4C0C2
:100A0000883709F4C7C08A3709F030C219C1898113
:100A100085FF05C084E793E064E771E054C0688116
:100A20008871883059F1893018F4882341F01EC24A
:100A3000803109F440C0883109F018C264C08AEFDF
:100A400092E00E94870902E00EC0FE01E00FF11D56
:100A500061816795662767958081680F8AEF92E0CC
:100A60000E94090A0E5F011780F38AEF92E00E944C
:100A70004C0A86E490E00E945712F8C19B818A815B
:100A8000163071F4979599279795980F4D81479552
:100A9000442747958C81480F862F692F70E008C046
:100AA000979599279795980F862F6FEF7FEF492F8E
:100AB0000E94E203DBC18091B80187303CF084E7FB
:100AC00093E060EA71E00E94E60ED0C18F5F8093F0
:100AD000B801992787FD9095FC01EE0FFF1FE80FE5
:100AE000F91FE15DFD4F60838B818795882787958E
:100AF0009A81890F81838D818795882787959C812D
:100B0000890F8283B3C15091B801151634F420E0E7
:100B1000C52FDD27C7FDD09511C08FEF8093B80199
:100B2000A5C1FC01EE0FFF1FE80FF91FE15DFD4FAE
:100B30006083662311F0422F24C02F5F822F90E044
:100B4000C817D90774F740E01CC04830C8F4C90181
:100B50000196D901AA0FBB1FA20FB31FA15DBD4F04
:100B6000FC01EE0FFF1FE80FF91FE15DFD4F8081D3
:100B70008C93808111968C931197828112968C931D
:100B80004F5F242F30E0C217D307FCF6515050932B
:100B9000B8016CC18981682F70E07695762F662741
:100BA000779567958881680F711D6115710521F032
:100BB000709369026093680280916702882309F04C
:100BC00055C10E94750352C1653008F44FC1F880C9
:100BD000C980EA80BB80DC808F2D82508C3008F089
:100BE00045C10F2D10E0C8010297EC01CC0FDD1FAD
:100BF000C80FD91FC659DD4FCE010E94C9078823EF
:100C000019F0CE010E945A074E2D50E05695542FF0
:100C10004427579547954C0D511D2D2D30E03695A5
:100C2000322F2227379527952B0D311DCE01B80184
:100C30000E9443088F2D64E070E00E94BE0116C13F
:100C4000623008F413C1898190E09695982F882727
:100C5000979587952881820F911D9093B701809376
:100C6000B6010A970CF002C18AE090E09093B701B8
:100C70008093B601FBC0623008F4F8C08981682F08
:100C800070E01230A1F08A8190E09695982F882725
:100C900097958795682B792B133049F02B81922FEC
:100CA0009295990F990F907C80E0682B792B888121
:100CB0000E948301DBC084E793E060EF0E940B0E8B
:100CC00084E793E06CE60E940B0E00E01EEF16C076
:100CD0001231A0F484E793E060E00E940B0E84E7F9
:100CE00093E061E00E940B0E84E793E061E00E94D4
:100CF0000B0E84E793E061E00E940B0E802F8E5074
:100D0000863050F484E793E062E00E940B0E84E7A3
:100D100093E06AE00E940B0E033051F0053041F081
:100D2000063031F0093021F00A3011F00B3051F467
:100D300084E793E063E00E940B0E84E793E068E0B1
:100D40000E940B0E1C3050F484E793E064E00E9494
:100D50000B0E84E793E06EE00E940B0E802F825111
:100D6000823050F484E793E066E00E940B0E84E743
:100D700093E061E00E940B0E84E793E06FE70E942E
:100D80000B0E0F5F1F5F043109F0A2CF6AC066230C
:100D900009F46CC0088184E793E060EF0E940B0EB9
:100DA00084E793E06EE60E940B0E84E793E0602FE9
:100DB0000E940B0E043108F054C0C02FD0E0FE0199
:100DC000E851FE4F84E793E060810E940B0E8E0194
:100DD000000F111F01501E4FF80160816F7784E7EB
:100DE00093E00E940B0EF80160817181CB01807845
:100DF000892B49F0660F672F661F770B6F7784E7A3
:100E000093E00E940B0ECC0FDD1FC150DE4F2881F6
:100E10003981C9018070907C892B19F1330F220B25
:100E2000330F322F221F622F6F7784E793E00E94E7
:100E30000B0E17C084E793E060EF0E940B0E84E76F
:100E400093E06AE60E940B0E02EF063010F06FE7A7
:100E500001C0602F84E793E00E940B0E0F5F063005
:100E6000A1F784E793E067EF0E940B0EDF91CF912B
:100E70001F910F91FF90EF90DF90CF90BF9008955A
:100E8000FC0180918E028C3090F482838F5F80937E
:100E90008E02815090E0FC01EE0FFF1FE80FF91F5A
:100EA000E157FD4F88EB9BE09283818308958FEF9C
:100EB00082830895DC0112968C91129790E0FC01D8
:100EC000EE0FFF1FE80FF91FE157FD4F80818F7B69
:100ED000808312968C916CE00E94631690E0AC01C6
:100EE000440F551F480F591F440F551F440F551FDE
:100EF00020E030E0C901840F951FFC01EE0FFF1FB9
:100F0000E80FF91FE157FD4F808186FD05C02F5F77
:100F10003F4F2C30310571F70895FC0122812C30B0
:100F2000B8F58081992787FD909548E850E0481BE7
:100F3000590B440F551F440F551F6417750784F054
:100F40008181992787FD909548E552E0481B590B10
:100F5000440F551F440F551F641775070CF4AB0160
:100F600042505040CA01AA2797FDA095BA2F880F7A
:100F7000991FAA1FBB1F4FB7F89430E0F901EE0F7D
:100F8000FF1FE20FF31FE157FD4F928381834FBF95
:100F90000895FC01828190E0FC01EE0FFF1FE80F35
:100FA000F91FE157FD4F8081829586958695817066
:100FB00009F081E00895AF92BF92CF92DF92EF9255
:100FC000FF920F931F93CF93DF93EC019B0182E07D
:100FD000603278070CF048C077FF03C020E030E0B3
:100FE00005C0653B710514F024EB30E000D000D063
:100FF000B901882777FD8095982F2881332727FD11
:101000003095E8E8AE2EB12CA21AB30AAA0CBB1C8C
:10101000AA0CBB1CCC24B7FCC094DC2CE981FF27B4
:10102000E7FDF09528E532E02E1B3F0B220F331F22
:10103000220F331F442737FD4095542FEDB7FEB7DD
:10104000218332834383548320E030E040E050E04A
:1010500004EBE02EF12C012D112D0E94FB159B01BC
:101060000F900F900F900F90CE01B9010E948D0745
:10107000DF91CF911F910F91FF90EF90DF90CF9074
:10108000BF90AF900895CF92DF92EF92FF921F939F
:10109000CF93DF93EC01162F7A0169018A818C309E
:1010A00008F064C0862F61E00E941E138A8190E0E0
:1010B000FC01EE0FFF1FE80FF91FE157FD4F1F73F3
:1010C0008081807C812B808380E292E08E199F0951
:1010D00064E070E00E946F16688380E699E08C19E6
:1010E0009D0964E070E00E946F166983AA818A2FCF
:1010F0006CE00E946316682F70E0AB01440F551F2F
:10110000460F571F440F551F440F551F20E030E076
:10111000C901840F951FFC01EE0FFF1FE80FF91F97
:10112000E157FD4F808186FD15C02F5F3F4F2C306A
:10113000310571F724C01092800082E08093810015
:101140001092850010928400B19A80916F008260A5
:1011500080936F008A2F90E0FC01EE0FFF1FE80FD5
:10116000F91FE157FD4F8081806480838A81DF9180
:10117000CF911F91FF90EF90DF90CF900895672B54
:10118000D1F2E8CF40E252E020E639E00E94430885
:1011900008951F920F920FB60F9211242F933F9331
:1011A0004F935F936F937F938F939F93AF93BF936F
:1011B000EF93FF938091B30287FF05C010928500E3
:1011C000109284002BC02091B302332727FD309565
:1011D00080918E0290E02817390704F58091B302C0
:1011E000992787FD9095FC01EE0FFF1FE80FF91F6F
:1011F000E157FD4F808186FF11C08091B30299278E
:1012000087FD9095FC01EE0FFF1FE80FF91FE157D6
:10121000FD4F80818F7360E00E945D138091B30267
:101220008F5F8093B3022091B302332727FD30955F
:1012300080918E0290E0281739070CF04EC0809103
:10124000B3028C300CF049C02091840030918500AD
:101250008091B302992787FD9095FC01EE0FFF1F47
:10126000E80FF91FE157FD4F81819281280F391F47
:1012700030938900209388008091B302992787FDDD
:101280009095FC01EE0FFF1FE80FF91FE157FD4F8E
:10129000808186FF2BC08091B302992787FD9095AE
:1012A000FC01EE0FFF1FE80FF91FE157FD4F808192
:1012B0008F7361E00E945D1319C080E49CE905C052
:1012C000809184009091850004969093890080938A
:1012D00088008FEF8093B30209C0809184009091C1
:1012E0008500049680549C4940F3EACFFF91EF912A
:1012F000BF91AF919F918F917F916F915F914F912E
:101300003F912F910F900FBE0F901F90189581E085
:101310008093F9026093D6021092F7021092F802BD
:1013200008952091D50230E08091D402281B310924
:10133000C90108954091D4028091D502481718F050
:101340002FEF3FEF0AC0E42FF0E0EC54FD4F808117
:10135000282F30E04F5F4093D402C9010895E091F7
:10136000D4028091D502E81718F0EFEFFFEF06C026
:10137000F0E0EC54FD4F8081E82FF0E0CF010895BC
:1013800008951092FD021092FC0288EE93E0A0E016
:10139000B0E08093FE029093FF02A0930003B0930D
:1013A000010384EC91E09093FB028093FA0208958C
:1013B000CF92DF92EF92FF920F931F93CF93DF9321
:1013C0007C016B018A018091F9028823A1F0C0E0C1
:1013D000D0E00DC0D701ED91FC91D601AC0FBD1F3F
:1013E0000190F081E02DC7016C9109952196C017FD
:1013F000D10780F304C0CB01642F0E940A0BC801FF
:10140000DF91CF911F910F91FF90EF90DF90CF90E0
:101410000895DF93CF930F92CDB7DEB7FC016983B8
:101420008091F9028823C9F08091F802803238F067
:1014300081E090E09383828320E030E015C08091CA
:10144000F702E82FF0E0E952FD4F998190838F5F1A
:101450008093F7028093F80205C0CE01019661E007
:101460000E940A0B21E030E0C9010F90CF91DF917B
:1014700008950F93062F8091D60267ED72E0409198
:10148000F80221E00E94B50A1092F7021092F802C9
:101490001092F9020F91089561E00E94390A0895AF
:1014A000413208F040E2862F64EB72E00E946C0A41
:1014B0001092D4028093D502089521E00E94500A30
:1014C00008951092D4021092D5021092F702109251
:1014D000F8020E94B60C0895382F413210F040E017
:1014E00042C0809106038823E1F791E090930603C0
:1014F000209308038FEF8093730310922E034150C3
:1015000040932F034F5F9093070380910703330F9E
:10151000832B8093070380910903813041F410925B
:101520000903809107038093BB0085EC01C085EE21
:101530008093BC00809106038130E1F380912E03FB
:10154000841710F440912E0320E030E00AC0FB0124
:10155000E20FF31FD901A25FBC4F8C9180832F5FF4
:101560003F4F2417A0F3842F08950F931F93582FF4
:10157000122F413210F081E04AC080910603882387
:10158000E1F782E080930603009308038FEF8093D6
:10159000730310922E0340932F03AEE0B3E0FB01E0
:1015A00002C081918D938E2F861B8417D0F31092E9
:1015B000070380910703550F852B809307038091C4
:1015C0000903813041F4109209038091070380934D
:1015D000BB0085EC01C085EE8093BC00112321F097
:1015E000809106038230E1F3809173038F3F11F401
:1015F00080E00DC080917303803211F482E007C057
:1016000080917303803311F084E001C083E01F9167
:101610000F910895482F613210F081E00895809174
:101620000603843011F082E0089560935103A0E333
:10163000B3E0842F9C01F90102C081918D938E2F1C
:10164000841B8617D0F380E008951F920F920FB687
:101650000F9211242F933F934F935F936F937F9338
:101660008F939F93AF93BF93EF93FF938091B900B4
:1016700090E0887F90708036910509F4F2C0813641
:101680009105CCF58832910509F47BC0893291052A
:10169000B4F48031910509F46FC0813191053CF4B7
:1016A000009709F447C1089709F04FC165C0883118
:1016B000910509F466C0809709F047C182C0803463
:1016C000910509F4A4C08134910544F48033910557
:1016D00009F482C0C89709F038C189C080359105E6
:1016E00009F489C08835910509F496C088349105BC
:1016F00009F02BC1AEC08839910509F413C18939AD
:101700009105ECF48837910509F4ABC08937910550
:101710004CF48836910509F4A4C08037910509F08E
:1017200014C19FC08838910509F4FCC08039910527
:1017300009F49DC08038910509F007C198C0803B2D
:10174000910509F4C6C0813B91054CF4803A91059E
:1017500009F49FC0883A910509F0F7C0BAC0803CEF
:10176000910509F4E3C0883C910509F4DFC0883B8A
:10177000910509F0EAC0C2C0809107038093BB00C5
:10178000CFC090912E0380912F03981768F4909109
:101790002E03E92FF0E0E25FFC4F80818093BB00D5
:1017A0009F5F90932E03BCC080910803882309F4A7
:1017B0004BC085ED8093BC008091BC0084FDFCCFC4
:1017C000C2C080E28093730385ED8093BC0080915A
:1017D000BC0084FDFCCFB7C080E38093730385ED2C
:1017E0008093BC008091BC0084FDFCCFACC088E33A
:1017F000809373039BC080912E039091BB00E82FD0
:10180000F0E0E25FFC4F90838F5F80932E03909116
:101810002E0380912F0382C080912E039091BB00F4
:10182000E82FF0E0E25FFC4F90838F5F80932E0300
:1018300080910803882341F085ED8093BC0080915E
:10184000BC0084FDFCCF7FC081E08093090384EA63
:101850006EC085ED8093BC008091BC0084FDFCCF00
:1018600072C083E0809306031092720359C0809186
:101870007203803208F056C0809172039091BB00D1
:10188000E82FF0E0EE5AFC4F90838F5F8093720355
:1018900047C080917203803230F4E0917203F0E02F
:1018A000EE5AFC4F108285ED8093BC008091BC0005
:1018B00084FDFCCF1092060360917203E0910C034B
:1018C000F0910D0382E593E070E0099510927203A8
:1018D0002DC084E0809306031092500310925103B0
:1018E000E0910A03F0910B0309958091510388233D
:1018F00029F481E0809351031092300390915003BA
:10190000E92FF0E0E05DFC4F80818093BB009F5F9A
:10191000909350039091500380915103981710F4C5
:1019200085EC01C085E88093BC000FC085EC8093F6
:10193000BC0009C01092730385ED8093BC008091B8
:10194000BC0084FDFCCF10920603FF91EF91BF9184
:10195000AF919F918F917F916F915F914F913F9147
:101960002F910F900FBE0F901F90189510920603A5
:1019700081E0809308031092090382E161E00E94F4
:101980005D1383E161E00E945D13E9EBF0E080818B
:101990008E7F808380818D7F808388E48093B800F0
:1019A00085E48093BC000895EF92FF920F931F93FC
:1019B0007C018B01DC01ED91FC91A081B1816F77FD
:1019C0002D913C91CF01F9010995D701ED91FC9141
:1019D000A081B181000F012F001F110B0F772D91F6
:1019E0003C91CF01602FF90109951F910F91FF9054
:1019F000EF900895FC010190F081E02DA081B1816C
:101A00002D913C91CF0160EFF90109950895FC01FA
:101A10000190F081E02DA081B1812D913C91CF0109
:101A200067EFF901099508950F931F938C01DC016D
:101A3000ED91FC91A081B1812D913C91CF0169EF95
:101A4000F9010995D801ED91FC91A081B1812D9109
:101A50003C91CF0162E0F9010995D801ED91FC912B
:101A6000A081B1812D913C91CF0163E0F9010995ED
:101A70001F910F9108951F93CF93DF93EC018A81FB
:101A80008823C9F1CE010E94FA0CE881F981A08176
:101A9000B1812D913C91CF0169E7F9010995E88168
:101AA000F981A081B1812B813C814D915C91CF0165
:101AB000F9016081FA010995E881F981A081B1817C
:101AC0002B813C814D915C91CF01F9016181FA013B
:101AD000099512E00AC0EB81FC81E10FF11D6081E4
:101AE000CE0170E00E94D40C1F5F8A81181798F312
:101AF000CE010E94070DDF91CF911F910895FC0147
:101B0000A081B181ED91FC9111970480F581E02DC8
:101B1000CD0109950895EF92FF920F931F938C01C9
:101B20007A01DC01ED91FC91A081B1816F70606E52
:101B30002D913C91CF01F9010995C801B7010E948F
:101B4000D40C1F910F91FF90EF900895EF92FF92A8
:101B50000F931F937C018A01DC01ED91FC91A08120
:101B6000B1816F7060692D913C91CF01F9010995A8
:101B7000D701ED91FC91A081B181602F6F772D91FC
:101B80003C91CF01F9010995D701ED91FC91A0811C
:101B9000B181000F012F001F110B2D913C91CF013E
:101BA000602FF90109951F910F91FF90EF90089513
:101BB000DF92EF92FF920F931F93CF93DF93EC018D
:101BC000162FD42E022FF32E0E94FA0CE881F981F1
:101BD000A081B1812D913C91CF01612FF90109952F
:101BE000202F3F2DC9017C0110E008C0F701619151
:101BF0007F01CE0170E00E94D40C1F5F1D15B0F371
:101C0000CE010E94070DDF91CF911F910F91FF90A0
:101C1000EF90DF900895FC010190F081E02DA0810C
:101C2000B1812D913C91CF01F90109950895FC01F5
:101C3000603DA9F0613D28F4603959F0603CA1F4A1
:101C40000BC0603E19F0643F79F40CC054A743A761
:101C5000089556A745A7089550AB47A7089552ABDE
:101C600041AB089554AB43AB0895FC016F3F11F4B1
:101C700056AB45AB0895FC0152AF41AF0895FC014E
:101C8000158216821782DC0180E018961C92189744
:101C90008F5F11968032C9F710A612A611A605A86B
:101CA000F6A9E02D309709F009950895FC011282FC
:101CB000148213820E943F0E089584E793E00E94ED
:101CC000560E08954F925F926F927F928F929F92DD
:101CD000AF92BF92CF92DF92EF92FF920F93DF937A
:101CE000CF9300D0CDB7DEB72B017A013A83298399
:101CF0008DE061E00E941E1300E089819A813C0121
:101D0000882477FC8094982C5701CC24B7FCC0948D
:101D1000DC2C11C0C401B3010E94FE118DE061E012
:101D20000E945D13C601B5010E94FE118DE060E0C6
:101D30000E945D130F5F802F90E08415950554F38A
:101D40000F900F90CF91DF910F91FF90EF90DF9068
:101D5000CF90BF90AF909F908F907F906F905F904B
:101D60004F9008950F931F938C018DE061E00E94C6
:101D70001E13C80162E070E048E250E022ED30E05E
:101D80000E94620E6AEF70E080E090E00E94FE1117
:101D9000C80163E070E048E250E022ED30E00E94CC
:101DA000620E6DE770E080E090E00E94FE111F91EE
:101DB0000F9108959A01FA0101900020E9F73197F7
:101DC000E41BF50B4E2F0E94D80D0895AB0161E77F
:101DD0000E94DA0E08951F93CF93DF93EC0188855C
:101DE000813731F0893789F5CE010E943B0D36C02D
:101DF0008FA998AD892B91F189A59AA5019762E0E9
:101E000070E00E946F16162F862F90E00E947310CC
:101E1000AC01DC0121E030E011C0FE01E20FF11D58
:101E200090859C932F5FFE01E20FF11D80858795C1
:101E300088278795890F8D932F5F3F5F311768F350
:101E4000EFA9F8ADCA01099509C0E9ADFAAD30971F
:101E500029F069A561502996AE010995DF91CF91CE
:101E60001F910895CF93DF93EC01A881B981ED9183
:101E7000FC9111970680F781E02DCD010995AC0109
:101E800088A5882391F0473F510529F418A6CE0173
:101E90000E94EB0E93C089A59AA5FE01E80FF91FD9
:101EA000408701969AA789A789C08D81882309F464
:101EB00046C0403851050CF042C081508D83FE0170
:101EC000E80FF11D4087882309F078C08E818823B0
:101ED00009F474C0803D49F1813D28F4803959F0FE
:101EE000803C59F51FC0803E19F0843F31F513C086
:101EF000EBA5FCA502C0EDA5FEA53097F1F0688525
:101F000070E07695762F6627779567958985680FB7
:101F1000711D8F8111C0EBA9FCA9309771F0688504
:101F2000898509C0EFA5F8A902C0E9A9FAA93097E7
:101F300021F068858F8170E009951E823FC0403F87
:101F4000510514F09A0106C09A01207F3070842F49
:101F50008F708F83203E3105F1F0213E310554F41E
:101F6000203C3105D1F0203D3105B9F02039310553
:101F700029F511C0243F310571F0253F310524F4C6
:101F8000203F3105D9F40DC0293F310599F02F3F8D
:101F90003105A1F40BC082E001C081E08D832E8366
:101FA0000DC081E088A71AA619A608C0CE010E941C
:101FB0003F0E04C084E793E00E94140DDF91CF919F
:101FC0000895AF92BF92CF92DF92EF92FF920F935C
:101FD0001F93CF93DF938C01D62EC72EB42EA22E43
:101FE000862F972F61EB71E00E94A900EC018D2DE7
:101FF0009C2D6FE270E00E949E00209779F07C019A
:102000000894E11CF11CE114F10441F09E012E5FE3
:10201000822F8E19D80112968C930FC0AD2DBC2D36
:10202000FD0101900020E9F7ED19EF5FD80112964C
:10203000EC932D2D3C2DC9017C01F8018381948105
:102040000E941011D80112968C9190E00E9473109A
:10205000FC01D80114969C938E93139712968C9141
:102060001297E80FF11D10821396ED91FC911497D1
:10207000B0821396ED91FC911497A18213968D91E5
:102080009C91149712964C9150E042505040029609
:10209000B7010E948F00DF91CF911F910F91FF90A8
:1020A000EF90DF90CF90BF90AF900895EF92FF92A6
:1020B0000F931F938C0130E4E32E34E0F32EC7011D
:1020C0000E943B14F801F182E082C8010E94B20E26
:1020D000C8010E94140DC8010E943B0D1F910F9171
:1020E000FF90EF9008950F931F93CF93DF93BC0160
:1020F0008230910510F462E070E0E0916404F091A8
:102100006504A0E0B0E040E050E024C0808191810F
:1021100086179707D0F08617970771F4828193810D
:10212000109729F013969C938E9312972CC090933E
:1021300065048093640427C04115510519F0841784
:10214000950718F4EF018D01AC01DF0182819381C5
:102150009C01F9013097D1F641155105F9F0CA01FA
:10216000861B970B8430910580F48A819B81011531
:10217000110521F0F8019383828304C090936504D4
:1021800080936404FE01329645C0FE01E80FF91FFA
:10219000619371930297998388833CC08091620414
:1021A00090916304892B41F48091BB019091BC0113
:1021B00090936304809362044091BD015091BE01ED
:1021C0004115510541F44DB75EB78091B901909129
:1021D000BA01481B590B2091620430916304241703
:1021E0003507B0F4CA01821B930B8617970780F05E
:1021F000AB014E5F5F4F8417950750F0420F531F9E
:102200005093630440936204F9016193719302C097
:10221000E0E0F0E0CF01DF91CF911F910F910895A1
:10222000CF93DF939C01009709F48FC0EC012297B4
:102230001B821A82609164047091650461157105B6
:1022400081F488819981820F931F209162043091DB
:1022500063042817390739F5D0936304C0936204E7
:1022600074C0DB0140E050E0AC17BD0708F1BB8350
:10227000AA83FE0121913191E20FF31FAE17BF0730
:1022800079F48D919C911197280F391F2E5F3F4F44
:102290003983288312968D919C9113979B838A830F
:1022A0004115510571F4D0936504C09364044DC089
:1022B00012968D919C911397AD01009711F0DC015E
:1022C000D3CFDA011396DC93CE931297FA012191C2
:1022D0003191E20FF31FCE17DF0769F488819981EE
:1022E000280F391F2E5F3F4FFA01318320838A81E7
:1022F0009B8193838283E0E0F0E0DB0112968D9175
:102300009C911397009719F0BC01FD01F6CFAB012A
:102310004E5F5F4FDB018D919C91840F951F209143
:102320006204309163042817390779F4309729F44F
:10233000109265041092640402C01382128242500B
:1023400050405093630440936204DF91CF9108950D
:102350001F920F920FB60F9211242F933F938F93DA
:102360009F93AF93BF938091B3039091B403A091D7
:10237000B503B091B6033091B7030196A11DB11D0D
:10238000232F2D5F2D3720F02D570196A11DB11D54
:102390002093B7038093B3039093B403A093B50342
:1023A000B093B6038091AF039091B003A091B103B5
:1023B000B091B2030196A11DB11D8093AF0390931C
:1023C000B003A093B103B093B203BF91AF919F91BB
:1023D0008F913F912F910F900FBE0F901F901895E6
:1023E0008FB7F8942091B3033091B4034091B503B3
:1023F0005091B6038FBFB901CA0108959B01AC018A
:102400007FB7F8948091AF039091B003A091B1038E
:10241000B091B20366B5A89B05C06F3F19F0019655
:10242000A11DB11D7FBFBA2FA92F982F8827860F16
:10243000911DA11DB11D62E0880F991FAA1FBB1F2E
:102440006A95D1F7BC012DC0FFB7F8948091AF0316
:102450009091B003A091B103B091B203E6B5A89BEF
:1024600005C0EF3F19F00196A11DB11DFFBFBA2FA6
:10247000A92F982F88278E0F911DA11DB11DE2E075
:10248000880F991FAA1FBB1FEA95D1F7861B970BD0
:10249000885E9340C8F2215030404040504068511F
:1024A0007C4F211531054105510571F608950197BD
:1024B00039F0880F991F880F991F02970197F1F73C
:1024C0000895789484B5826084BD84B5816084BDAC
:1024D00085B5826085BD85B5816085BDEEE6F0E09D
:1024E000808181608083E1E8F0E0108280818260F9
:1024F0008083808181608083E0E8F0E0808181607A
:102500008083E1EBF0E0808184608083E0EBF0E0A9
:10251000808181608083EAE7F0E08081846080834D
:1025200080818260808380818160808380818068F7
:1025300080831092C1000895982F8E3008F09E502D
:1025400097708091BF018295880F880F807C892BBE
:1025500080937C0080917A00806480937A008091DF
:102560007A0086FDFCCF2091780040917900942F6D
:1025700080E030E0282B392BC90108951F93CF93B9
:10258000DF93182FEB0161E00E941E13209709F4DE
:102590004AC0CF3FD10509F449C0E12FF0E0E25530
:1025A000FF4F84918330C1F0843028F4813051F0A2
:1025B0008230B1F50CC0863019F1873049F1843092
:1025C00079F514C084B5806884BDC7BD33C084B5B7
:1025D000806284BDC8BD2EC08091800080688093D9
:1025E0008000D0938900C093880024C0809180002F
:1025F000806280938000D0938B00C0938A001AC0C1
:102600008091B00080688093B000C093B30012C086
:102610008091B00080628093B000C093B4000AC083
:10262000C038D1051CF4812F60E002C0812F61E029
:102630000E945D13DF91CF911F910895CF93DF9397
:10264000482F50E0CA0186569F4FFC0134914A57EB
:102650005F4FFA018491882369F190E0880F991FF8
:10266000FC01E859FF4FA591B491FC01EE58FF4FD2
:10267000C591D491662351F42FB7F8948C91932F80
:10268000909589238C93888189230BC0623061F4F3
:102690002FB7F8948C91932F909589238C938881F0
:1026A000832B88832FBF06C09FB7F8948C91832B10
:1026B0008C939FBFDF91CF910895482F50E0CA01BE
:1026C00082559F4FFC012491CA0186569F4FFC0101
:1026D00094914A575F4FFA013491332309F440C073
:1026E000222351F1233071F0243028F42130A1F05D
:1026F000223011F514C02630B1F02730C1F024305B
:10270000D9F404C0809180008F7703C0809180004D
:102710008F7D8093800010C084B58F7702C084B510
:102720008F7D84BD09C08091B0008F7703C08091F8
:10273000B0008F7D8093B000E32FF0E0EE0FFF1F1D
:10274000EE58FF4FA591B4912FB7F894662321F46A
:102750008C919095892302C08C91892B8C932FBFEB
:10276000089508951F920F920FB60F9211242F9380
:102770003F934F938F939F93EF93FF938091C0006C
:1027800082FD1DC04091C6002091F8033091F903ED
:102790002F5F3F4F2F7330708091FA039091FB03AE
:1027A0002817390771F0E091F803F091F903E85424
:1027B000FC4F40833093F9032093F80302C08091CB
:1027C000C600FF91EF919F918F914F913F912F9173
:1027D0000F900FBE0F901F901895E0914C04F09150
:1027E0004D04E05CFF4F8191919120813181821BEA
:1027F000930B8F739070892B11F00E94B113089581
:102800001F920F920FB60F9211242F933F938F9325
:102810009F93EF93FF9320913C0430913D0480916E
:102820003E0490913F042817390731F48091C1008C
:102830008F7D8093C10014C0E0913E04F0913F046D
:10284000E450FC4F208180913E0490913F0401961A
:102850008F73907090933F0480933E042093C60042
:10286000FF91EF919F918F913F912F910F900FBE0C
:102870000F901F901895AF92BF92DF92EF92FF9248
:102880000F931F93CF93DF93EC017A018B01DD242B
:10289000403081EE580780E0680780E0780711F04B
:1028A000DD24D39491E0A92EB12CEC89FD89DD20A3
:1028B00069F0C50108A002C0880F991F0A94E2F7C9
:1028C000808360E079E08DE390E005C0108260E8ED
:1028D00074E88EE190E0A80197010E9482162150D1
:1028E000304040405040569547953795279580E1B8
:1028F0002030380720F0DD2011F0DD24D6CFE88924
:10290000F9893083EA89FB89208319A2EE89FF893E
:10291000408121E030E0C9010C8C02C0880F991F72
:102920000A94E2F7482B4083EE89FF894081C90170
:102930000D8C02C0880F991F0A94E2F7482B408340
:10294000EE89FF894081C9010E8C02C0880F991F52
:102950000A94E2F7482B4083EE89FF8980810F8C2F
:1029600002C0220F331F0A94E2F720952823208308
:10297000DF91CF911F910F91FF90EF90DF90BF906B
:10298000AF900895DC011C96ED91FC911D97E05CE1
:10299000FF4F2191319180819181281B390B2F7339
:1029A0003070C9010895DC011C96ED91FC911D97D2
:1029B000E05CFF4F20813181E054F040DF01AE5BED
:1029C000BF4F8D919C9111972817390719F42FEF5C
:1029D0003FEF07C08D919C91E80FF91F8081282F50
:1029E00030E0C9010895DC011C96ED91FC911D9722
:1029F000E05CFF4F20813181E054F040DF01AE5BAD
:102A0000BF4F8D919C9111972817390719F42FEF1B
:102A10003FEF10C08D919C911197E80FF91F208115
:102A20008D919C91119701968F73907011969C9344
:102A30008E9330E0C9010895DC0191968C919197B5
:102A4000882339F05496ED91FC915597808186FF4B
:102A5000F9CF91961C920895CF93DF93EC01EE8508
:102A6000FF85E05CFF4F20813181E054F0402F5F13
:102A70003F4F2F733070DF01AE5BBF4F8D919C9144
:102A8000119728173907D1F3E05CFF4F80819181BE
:102A9000E054F040E80FF91F6083EE85FF85E05CAD
:102AA000FF4F31832083EE89FF89208181E090E010
:102AB0000F8C02C0880F991F0A94E2F7282B2083FD
:102AC00081E089A3EC89FD8980818064808381E035
:102AD00090E0DF91CF910895109243041092420448
:102AE00088EE93E0A0E0B0E0809344049093450426
:102AF000A0934604B093470484ED91E09093410481
:102B00008093400488EB93E090934D0480934C04B1
:102B10008CEF93E090934F0480934E0485EC90E00B
:102B2000909351048093500484EC90E0909353046C
:102B30008093520480EC90E0909355048093540469
:102B400081EC90E0909357048093560482EC90E0DF
:102B5000909359048093580486EC90E090935B0422
:102B600080935A0484E080935C0483E080935D0446
:102B700087E080935E0485E080935F0481E080932A
:102B800060040895CF93DF930E9461120E94340382
:102B9000CDEED3E10E944C042097E1F30E94ED13A7
:102BA000F9CFCF92DF92EF92FF920F931F93CF93C3
:102BB000DF937C016B018A01C0E0D0E00FC0D60139
:102BC0006D916D01D701ED91FC910190F081E02DA7
:102BD000C7010995C80FD91F0150104001151105F3
:102BE00071F7CE01DF91CF911F910F91FF90EF9080
:102BF000DF90CF9008952F923F924F925F926F9205
:102C00007F928F929F92AF92BF92CF92DF92EF927C
:102C1000FF920F931F93DF93CF93CDB7DEB73B01A6
:102C20004C0119012A016D897E898F89988D6A1955
:102C30007B098C099D09621A730A840A950AA4010A
:102C400093010E944416E218F30804091509A8012B
:102C500097010E94A4162A0D3B1D4C1D5D1DB90154
:102C6000CA01CF91DF911F910F91FF90EF90DF90FC
:102C7000CF90BF90AF909F908F907F906F905F901C
:102C80004F903F902F900895629FD001739FF00165
:102C9000829FE00DF11D649FE00DF11D929FF00DEC
:102CA000839FF00D749FF00D659FF00D9927729F23
:102CB000B00DE11DF91F639FB00DE11DF91FBD01AE
:102CC000CF0111240895991B79E004C0991F96172C
:102CD00008F0961B881F7A95C9F78095089597FB91
:102CE000092E07260AD077FD04D049D006D000204F
:102CF0001AF4709561957F4F0895F6F79095819538
:102D00009F4F0895A1E21A2EAA1BBB1BFD010DC007
:102D1000AA1FBB1FEE1FFF1FA217B307E407F5078B
:102D200020F0A21BB30BE40BF50B661F771F881F67
:102D3000991F1A9469F760957095809590959B01FD
:102D4000AC01BD01CF01089597FB092E05260ED0D9
:102D500057FD04D0D7DF0AD0001C38F450954095B9
:102D6000309521953F4F4F4F5F4F0895F6F790955F
:102D70008095709561957F4F8F4F9F4F0895AA1B47
:102D8000BB1B51E107C0AA1FBB1FA617B70710F056
:102D9000A61BB70B881F991F5A95A9F78095909588
:102DA000BC01CD010895EE0FFF1F0590F491E02DB9
:062DB0000994F894FFCF26
:102DB600556E6B6E6F776E2070696E206D6F6465F1
:102DC600005374616E646172644669726D61746108
:102DD6002E696E6F00493243205265616420457248
:102DE600726F723A20546F6F206D616E792062792E
:102DF600746573207265636569766564004932435C
:102E06002052656164204572726F723A20546F6F6A
:102E160020666577206279746573207265636569DB
:102E26007665640031302D62697420616464726570
:102E36007373696E67206D6F6465206973206E6FAA
:102E4600742079657420737570706F727465640090
:102E5600746F6F206D616E79207175657269657327
:102E6600002E637070001300FF80006604000001EE
:102E760000000000090AD80991099A09AF09C0099A
:102E8600000000002C15D115C214F314D3141C1520
:00000001FF
